:1000000012C02CC02BC02AC029C028C027C026C0BF
:1000100025C078C123C033C054C020C01FC01EC03B
:100020001DC01CC01BC011241FBECFE5D4E0DEBF25
:10003000CDBF12E0A0E6B0E0E2E1F5E102C005903C
:100040000D92AE39B107D9F713E0AEE9B2E001C0C5
:100050001D92A431B107E1F7EAD459CAD1CF90BDBE
:1000600089B988E18AB986E880BD1092A102109210
:10007000A0021092E3021092E202579A08951F9292
:100080000F920FB60F9211242F938F939F93EF939C
:10009000FF939CB18091A0028F5F81708093A0023A
:1000A0002091A102EEE9F2E0E80FF11D9083FF91AB
:1000B000EF919F918F912F910F900FBE0F901F90F6
:1000C00018951F920F920FB60F9211248F939F9342
:1000D000EF93FF939091E2028091E302981761F011
:1000E000E091E302EF5FEF73E093E302F0E0EE559F
:1000F000FD4F80818CB901C05598FF91EF919F9180
:100100008F910F900FBE0F901F9018959091A002A5
:100110008091A10220E0981321E0822F0895909110
:10012000A0028091A1029817D1F3E091A102EF5FA4
:10013000E170E093A102F0E0E256FD4F8081089566
:10014000282F9091E2029F5F9F738091E30298179E
:10015000E1F3E92FF0E0EE55FD4F20839093E202AA
:10016000559A08951F93CF93DF93EC0197FF08C032
:100170008DE2E6DFD095C195DF4F02C0C051D74276
:1001800027E2C031D207D4F702C0C85ED34033E0C3
:10019000C83ED307D4F790E002C0C456D040892FA0
:1001A0009F5FC436D105CCF790E001C02A97192F84
:1001B0009F5FCA30D105D4F7805DC2DF812F805D9B
:1001C000BFDF9E01205D822FBBDFDF91CF911F91AA
:1001D0000895EF92FF920F931F93CF93DF93EC015B
:1001E00097FD02C090E004C0D095C195DF4F9FEF0E
:1001F00080E002C0C051D742E82E8F5F27E2C031B5
:10020000D207C4F780E002C0C85ED340F82E8F5FEB
:1002100033E0C83ED307C4F780E002C0C456D040E4
:10022000082F8F5FC436D105CCF780E001C02A9734
:10023000182F8F5FCA30D105D4F7992311F08DE2C2
:1002400001C080E27DDF8E2D805D7ADF8F2D805DA5
:1002500077DF802F805D74DF812F805D71DF9E01ED
:10026000205D822F6DDFDF91CF911F910F91FF9065
:10027000EF9008951F93CF93DF93182FC0E0D0E045
:10028000812F881F8827881F805D5ADF2196C830FC
:10029000D10511F0110FF4CFDF91CF911F91089587
:1002A0000F931F93182F882311F020E003C080E3E1
:1002B00019C01456322F2F5F812F90E0843691059C
:1002C000C4F720E001C01A50022F2F5F812F90E069
:1002D0000A97CCF7832F805D33DF802F805D30DF7E
:1002E000812F805D2DDF1F910F910895CF93DF93B4
:1002F000EC0102C025DF219688818823D9F7DF91A0
:10030000CF9108951F920F920FB60F9211245F9311
:100310006F937F938F939F93AF93BF9380911103BC
:100320009091120301969093120380931103809190
:1003300011039091120362E370E09ED8892B19F4A7
:1003400081E080931303BF91AF919F918F917F9133
:100350006F915F910F900FBE0F901F9018951092A4
:100360001203109211031092130383B7836083BFAB
:1003700012BE89B7816089BF089589B78E7F89BF12
:10038000109212031092110389B7816089BF0895FA
:1003900089B7816089BF089589B78E7F89BF089525
:1003A000E199FECF9FBB8EBB6DBBF894E29AE19AB8
:1003B00078940895E199FECF9FBB8EBBE09A8DB3F0
:1003C0000895E4EEF2E080E991E08193919322E0D8
:1003D000E43FF207D1F786E086B983E487B9379A1C
:1003E000369A0895369921C047B14770E42FF0E05E
:1003F00064B175B1EE0FFF1FEC51FD4F20813181CB
:10040000C901880F991F820F931F860F971F96951A
:10041000879596958795918380834F5F483009F43F
:1004200043E04770406447B9369A0895883018F021
:10043000E0E0F0E009C0E82FF0E0EE0FFF1FEC5124
:10044000FD4F0190F081E02DCF010895382F6623F4
:1004500061F422B381E090E002C0880F991F3A95C1
:10046000E2F78095822382BB089522B381E090E079
:1004700002C0880F991F3A95E2F7282B22BB0895F6
:100480008F929F92AF92BF92CF92DF92EF92FF92A4
:100490000F931F93CF93DF934B0100917001109145
:1004A0007101EC01081719070CF4E801A0906E0126
:1004B000B0906F01BE01882777FD8095982F95D564
:1004C0006B017C011C161D0634F4B801882777FDEA
:1004D0008095982F05C0B501882777FD8095982FC6
:1004E00084D59B01AC01C701B601DAD47B018C0134
:1004F000B401882777FD8095982F77D59B01AC01B3
:10050000C801B701D8D3CBD5CB01DF91CF911F91D3
:100510000F91FF90EF90DF90CF90BF90AF909F90A2
:100520008F900895CF93DF93EC0127DF8091110323
:10053000909112038C179D07C8F31FDFDF91CF91B5
:100540000895CF93DF93EC012091110330911203B2
:10055000999B03C08AEF90E002C084E690E0821786
:10056000930778F40ADF8881882329F4929881E040
:100570008883939A06C0929A8091FB028111939886
:100580001882DF91CF9108951F93182F80E690E095
:10059000ADDE812F805DD4DD80E2D2DD1F91089534
:1005A000EF92FF921F93CF93DF937C01EB0110E05A
:1005B000812FEADF83E690E099DE209719F487E641
:1005C00090E00CC08DE690E091DECE018FDEC70199
:1005D000C9DD812F805DB4DD82E790E087DE1F5F9B
:1005E000163031F7DF91CF911F91FF90EF90089572
:1005F000EF92FF920F931F93CF93DF93062F7A0111
:10060000E901182F15C0812FBFDF83E690E06EDE71
:10061000209719F487E690E009C08DE690E066DE49
:10062000CE0164DEC7019EDD82E790E05FDE1F5FE2
:1006300010174CF3DF91CF911F910F91FF90EF9026
:100640000895FF920F931F93162FF42E022F9CDF15
:1006500089E790E04BDE1F3F19F0812F805D70DD50
:100660008F2D6EDD0F3F11F0802F1ADE8CE790E0AA
:100670003DDE1F910F91FF900895EF92FF920F932F
:100680001F93E82E989903C010E006E004C0109173
:100690000003012F0F5F8E2D80958623F82E81FF9A
:1006A00013C0E2FE09C08091FD028F5F8093FD02BE
:1006B000803110F01092FD024091FD022FE730E0F2
:1006C00050E0602F812F94DFF0FE13C0E2FE09C0DE
:1006D0008091FE028F5F8093FE02803110F01092B5
:1006E000FE024091FE0221E830E050E0602F812FB1
:1006F0007FDFF3FE30C0E2FC0DC020E046E56FEF87
:10070000809100039EDF2FEF46E46FEF809100039E
:1007100098DF21C0989918C08091FF0280FF05C022
:1007200060E070E080E090E004C063E870E08695EF
:1007300090E036DF8091FF028F5F8093FF0280316F
:1007400050F01092FF0207C020E030E040E050E09F
:10075000602F812F4DDFF5FE1EC08091000314DF56
:1007600085E890E0C3DD809100030EDF8CE890E027
:10077000BDDD8091000308DF83E990E0B7DD22E36F
:1007800044E56FEF809100035CDF2FEF43E46FEFF0
:100790008091000356DFF4FE20C080910003F4DE58
:1007A0008DE990E0A3DD8E2D90E0809590958C7082
:1007B00090708830910541F08C30910541F004979C
:1007C00049F484EA90E008C088EA90E005C08CEA29
:1007D00090E002C080EB90E089DD1F910F91FF90C7
:1007E000EF900895FF920F931F93CF93DF93F82E0E
:1007F000062FEA01122F2F3F09F41EEF8F2DC4DEC2
:1008000089E790E073DD0F3F19F0802F805D98DC61
:1008100088E496DCCE01A6DC8CE790E067DD212F32
:1008200046E5602F8F2D0DDF2FEF46E4602F8F2DD3
:1008300008DFDF91CF911F910F91FF9008951F93D3
:10084000CF93DF93EC01CB0164E170E019DE2091DE
:10085000F5023091F602280F391F3093F6022093EB
:10086000F50281E02936380734F0285631403093BC
:10087000F6022093F5028091F5029091F60297FF1F
:1008800006C088599E4F9093F6028093F50261EF5F
:100890007FEFCE01F5DD2091F4022091F702309137
:1008A000F802280F391F3093F8022093F7022E3FE9
:1008B000310534F08EEF90E09093F8028093F702C8
:1008C0008091F7029091F802029724F41092F802B6
:1008D0001092F70298990EC010E04091F5025091E5
:1008E000F6022091F7026FEF812F7CDF1F5F163039
:1008F000A1F70AC04091F5025091F6022091F7024B
:100900006FEF809100036EDFDF91CF911F9108950B
:10091000FF920F931F93CF93DF93082F162FF42E80
:1009200022E344E58EDECF2DD0E0FE01EE58FE4FEF
:10093000208142E5612F802F84DEFE01E658FE4FC4
:10094000208147E4612F802F7CDECE57DE4F288147
:1009500042E4612F802F75DE2FEF46E4612F802F58
:1009600070DEDF91CF911F910F91FF9008951F933B
:1009700080EC87BB8FE388BB14BA87E085BB8EE031
:1009800081BB80EF82BB8BE090E069DB1ADDE7DCA6
:10099000789480B390E080959095807F907024E06B
:1009A000959587952A95E1F78F70809300032CE346
:1009B0008202900111242C5E3F4F3093F602209367
:1009C000F5028FE790E09093F8028093F70284EBB2
:1009D00090E08CDC2091F50248E46FEF80910003F9
:1009E00030DE2091F70246E56FEF8091000329DEAB
:1009F0002FEF46E46FEF8091000323DE10E009C083
:100A0000939884E690E08EDD939A84E690E08ADD08
:100A10001F5F212F30E080910003992787FD90957B
:100A2000281739076CF3939A929A1F9108957F9231
:100A30008F929F92AF92BF92CF92DF92EF92FF92EE
:100A40000F931F93DF93CF930F92CDB7DEB7198229
:100A50008EDF51E0C52E53E0D52EF6011192119292
:100A600023E0E131F207D1F7AA24BB2420C0BADC8D
:100A70000F5F1F4F3FE100341307C9F7F7010081F3
:100A80001181892DD3DC080F191FF70101931193F0
:100A90007F019394F8E09F1619F000E010E0E7CF93
:100AA0000894A11CB11C28E0A216B10431F041E069
:100AB000E42E43E0F42E9924F0CFF6018081918159
:100AC00033E0969587953A95E1F7819391936F017D
:100AD000F1E1CF16F3E0DF0681F74E010894811CA7
:100AE000911C772473947EDCC4012BDD8091130369
:100AF0008823C9F31092130383E098DC895D934047
:100B00001CF07092FB0202C01092FB0285E08EDCAA
:100B100020910B0330910C035C01A21AB30A80915F
:100B20008C0190918D01F501E81BF90BCF01F7FFC6
:100B300003C0909581959F4F06970CF1809100031B
:100B400023DD82EC90E0D2DB9501B7FE04C02227C2
:100B500033272A193B0980918A0190918B0128172C
:100B600039071CF480E3ECDA07C0609168017091EA
:100B70006901C50185DCF6DA85EC90E0B7DBB0925F
:100B80008D01A0928C0184E051DC20910903309109
:100B90000A038C01021B130B80918E0190918F012F
:100BA0009801281B390BC90137FF03C09095819527
:100BB0009F4F069784F180910003E6DC8BEC90E078
:100BC00095DB980117FF04C022273327201B310B28
:100BD00080918A0190918B01281739071CF480E3DA
:100BE000AFDA16C099990AC060916C0170916D01DD
:100BF000709561957F4FC80143DC09C060916A011F
:100C000070916B01709561957F4FC80139DCAADA4C
:100C100085EC90E06BDB10938F0100938E0186E0F2
:100C200005DC20910D0330910E036C01C21AD30A2A
:100C300087E0FCDB20910F03309110037C01E21A66
:100C4000F30A8091F4028823A1F08EEC90E04EDB51
:100C5000C80188DA83ED90E049DBC50183DA87EDCE
:100C600090E044DBC6017EDA8BED90E03FDBC7010C
:100C700079DAC601D7FE04C0882799278C199D0907
:100C80000B974CF4C701F7FE04C0882799278E19EB
:100C90009F090B971CF0B601C701D1DD16B3609117
:100CA0009401161711F0812FE8DC1093940183B39F
:100CB0008091F40218CFA0E2B0E0E0E6F6E0F0C3E5
:100CC00069837A838B839C832D833E834F835887EC
:100CD000BE01675F7F4FCE01019656D3BE016F5EA6
:100CE0007F4FCE01059650D39985923088F089893F
:100CF0008230C8F0943019F4823051F404C084304A
:100D000029F4923081F485E991E0C6C0923049F42B
:100D100020E09A858A89981321E02A87CE010996D6
:100D2000BBC0823049F420E09A858A89981321E07B
:100D30002A8BCE014196B0C02D843E844F845888C2
:100D40006D887E888F88988CEE24FF248701AA24E2
:100D5000BB24650140E050E060E070E0E0E0F0E0DE
:100D6000C10181709070892BE9F0E60CF71C081D19
:100D7000191D9A01AB012A0D3B1D4C1D5D1D80E024
:100D800090E0A0E0B0E0E614F7040805190520F4AF
:100D900081E090E0A0E0B0E0BA01A901480F591F3E
:100DA0006A1F7B1FAA0CBB1CCC1CDD1C97FE08C055
:100DB00081E090E0A0E0B0E0A82AB92ACA2ADB2AA4
:100DC0003196E032F10549F0660C771C881C991CBD
:100DD0005694479437942794C3CFFA85EA892B8990
:100DE0003C898B859C85280F391F2E5F3F4F17C08C
:100DF000CA0181709070892B61F016950795F79460
:100E0000E79480E090E0A0E0B0E8E82AF92A0A2B15
:100E10001B2B76956795579547952F5F3F4F77FD2D
:100E2000E7CF0CC0440F551F661F771F17FD4160A9
:100E3000EE0CFF1C001F111F21503040403090E08D
:100E4000590790E0690790E4790760F32B8F3C8F96
:100E5000DB01CA018F779070A070B070803491056B
:100E6000A105B10561F447FD0AC0E114F1040105D3
:100E7000110529F0405C5F4F6F4F7F4F40781A8E0D
:100E8000FE1711F081E08A8F4D8F5E8F6F8F78A3F0
:100E900083E0898FCE014996A2D1A096E2E11CC3DE
:100EA000A8E1B0E0E5E5F7E003C369837A838B83CB
:100EB0009C832D833E834F835887B9E0EB2EF12C22
:100EC000EC0EFD1EB701CE0101965ED28E010F5EC3
:100ED0001F4FB801CE01059657D22985223008F45C
:100EE0007CC03989323010F4B8017AC08A859A8979
:100EF00089278A87243011F0223031F4231709F032
:100F00006CC065E971E06CC0343039F41D861E8612
:100F10001F86188A1C861B8604C0323021F484E0A8
:100F20008987B7015DC02B853C858B899C89281BEF
:100F3000390B3C872B87ED84FE840F851889AD889B
:100F4000BE88CF88D88CEA14FB040C051D0540F43C
:100F5000EE0CFF1C001F111F215030403C872B87D7
:100F600020E030E040E050E080E090E0A0E0B0E43D
:100F70006FE170E0EA14FB040C051D0540F0282B1E
:100F8000392B4A2B5B2BEA18FB080C091D09B69577
:100F9000A79597958795EE0CFF1C001F111F6150B8
:100FA000704041F7DA01C9018F779070A070B0707E
:100FB00080349105A105B10561F427FD0AC0E11453
:100FC000F1040105110529F0205C3F4F4F4F5F4FA1
:100FD00020782D873E874F87588BBE01675F7F4FF4
:100FE000CB01FDD06896EAE07FC2A8E0B0E0EAEF6E
:100FF000F7E05FC29B01AC0183E08983DA01C9019C
:101000008827B7FD83959927AA27BB27B82E2115D6
:1010100031054105510519F482E0898339C08823DF
:10102000A9F0203080E0380780E0480780E85807C2
:1010300029F460E070E080E09FEC2EC0EE24FF24F5
:101040008701E21AF30A040B150B02C079018A0129
:101050008EE1C82ED12CDC82CB82ED82FE820F8302
:101060001887C801B7016CD001971816190684F4C7
:10107000082E04C0EE0CFF1C001F111F0A94D2F7AB
:10108000ED82FE820F831887C81AD90ADC82CB82D0
:10109000BA82CE010196A3D02896E9E026C2ACE040
:1010A000B0E0E4E5F8E00CC269837A838B839C832B
:1010B000BE016B5F7F4FCE01019666D18D8182307C
:1010C00061F1823050F1843021F48E81882351F116
:1010D0002EC02F81388537FD20C06E812F3131051C
:1010E0001CF06623F9F023C08EE190E0821B930B85
:1010F00029853A854B855C8504C05695479537957B
:1011000027958A95D2F76623B1F050954095309592
:1011100021953F4F4F4F5F4F0EC020E030E040E041
:1011200050E009C02FEF3FEF4FEF5FE704C020E032
:1011300030E040E050E8B901CA012C96E2E0DCC1A1
:10114000EF92FF920F931F937B018C0180E0E816D2
:1011500080E0F80681E0080780E0180788F48FEF48
:10116000E816F1040105110531F028F088E090E05F
:10117000A0E0B0E017C080E090E0A0E0B0E012C0D6
:1011800080E0E81680E0F80680E0080781E01807B4
:1011900028F088E190E0A0E0B0E004C080E190E0B9
:1011A000A0E0B0E020E230E040E050E0281B390B46
:1011B0004A0B5B0B04C016950795F794E7948A9544
:1011C000D2F7F701E356FE4F8081281B3109410910
:1011D0005109C9011F910F91FF90EF900895DF927F
:1011E000EF92FF920F931F93FC01E480F58006813C
:1011F0001781D1808081823048F480E090E0A0E1C6
:10120000B0E0E82AF92A0A2B1B2BA5C0843009F488
:101210009FC0823021F4EE24FF24870105C0E11431
:10122000F1040105110519F4E0E0F0E096C06281D7
:1012300073819FEF623879070CF05BC022E83FEFC3
:10124000261B370B2A3131052CF020E030E040E03E
:1012500050E02AC0B801A701022E04C07695679518
:10126000579547950A94D2F781E090E0A0E0B0E06E
:1012700004C0880F991FAA1FBB1F2A95D2F7019798
:10128000A109B1098E219F21A023B1230097A105B7
:10129000B10521F081E090E0A0E0B0E09A01AB015F
:1012A000282B392B4A2B5B2BDA01C9018F779070E1
:1012B000A070B07080349105A105B10539F427FF05
:1012C00009C0205C3F4F4F4F5F4F04C0215C3F4F30
:1012D0004F4F5F4FE0E0F0E02030A0E03A07A0E0A1
:1012E0004A07A0E45A0710F0E1E0F0E079018A0132
:1012F00027C06038710564F5FB01E158FF4FD80144
:10130000C7018F779070A070B07080349105A105EF
:10131000B10539F4E7FE0DC080E490E0A0E0B0E054
:1013200004C08FE390E0A0E0B0E0E80EF91E0A1FD1
:101330001B1F17FF05C016950795F794E794319684
:1013400087E016950795F794E7948A95D1F705C03D
:10135000EE24FF248701EFEFF0E06E2F67956627FC
:101360006795902F9F77D794DD24D7948E2F8695FD
:10137000492F462B582F5D29B701CA011F910F91A4
:10138000FF90EF90DF900895FC01DB0140815181D7
:101390002281622F6F7770E0221F2227221F938104
:1013A000892F880F822B282F30E0991F9927991FAA
:1013B00011969C93119721153105A9F541155105F9
:1013C0006105710511F482E037C082E89FEF139642
:1013D0009C938E9312979A01AB0167E0220F331F03
:1013E000441F551F6A95D1F783E08C930DC0220FDF
:1013F000331F441F551F12968D919C91139701978F
:1014000013969C938E931297203080E0380780E0EB
:10141000480780E4580758F314962D933D934D9355
:101420005C93179708952F3F310579F441155105C5
:101430006105710519F484E08C93089564FF03C07D
:1014400081E08C9312C01C9210C02F57304013962D
:101450003C932E93129783E08C9387E0440F551FA3
:10146000661F771F8A95D1F7706414964D935D932C
:101470006D937C9317970895AA1BBB1B51E107C07E
:10148000AA1FBB1FA617B70710F0A61BB70B881F14
:10149000991F5A95A9F780959095BC01CD010895A3
:1014A0002F923F924F925F926F927F928F929F9274
:1014B000AF92BF92CF92DF92EF92FF920F931F9362
:1014C000CF93DF93CDB7DEB7CA1BDB0B0FB6F89413
:1014D000DEBF0FBECDBF09942A88398848885F8453
:1014E0006E847D848C849B84AA84B984C884DF80C4
:1014F000EE80FD800C811B81AA81B981CE0FD11DA8
:101500000FB6F894DEBF0FBECDBFED010895F8947D
:02151000FFCF0B
:101512007B36003C4D20005653543E7D00565046CB
:1015220020002E6D70333E7D003C4C003E7D0068F5
:101532000061007300247030302A7D002473303043
:101542002A7D005B48414C5420305D7D005B4D4F4D
:1015520044452000315D7D00325D7D00335D7D00BC
:10156200305D7D0052656D6F74652076312E330DCE
:101572000A002473002A7D0A0D20002470000A0D3F
:10158200443A0020533A0020483A0020563A000CD0
:101592000030303230383037320030303638313780
:1015A200323700303233353534383200303531326B
:1015B200363034350030363937333038370031334E
:1015C2003533343835310033373535383538003135
:1015D20031393039323932003037383633363231F8
:1015E20000303838353737383800303939333939FF
:1015F2003638003139393836333834000000E100EA
:10160200EA00F300FC0005010E0117011F01280189
:1016120031013A0143014C0164003C005000F401E5
:10162200F401FE0000FEFE00FE0000FE0000FEFED1
:10163200FE000000FEFE00FEFE0003009CFF9CFF79
:101642009CFF9CFFFF000000000000000000010260
:10165200020303030304040404040404040505054B
:101662000505050505050505050505050506060625
:101672000606060606060606060606060606060608
:1016820006060606060606060606060606070707F5
:1016920007070707070707070707070707070707D8
:1016A20007070707070707070707070707070707C8
:1016B20007070707070707070707070707070707B8
:1016C20007070707070707070707070707080808A5
:1016D2000808080808080808080808080808080888
:1016E2000808080808080808080808080808080878
:1016F2000808080808080808080808080808080868
:101702000808080808080808080808080808080857
:101712000808080808080808080808080808080847
:101722000808080808080808080808080808080837
:101732000808080808080808080808080808080827
:0E174200080808080808080808080808080031
:00000001FF
